:1000000083160030850080308600843081008312A2
:1000100007309F00850186018B01FF30B300AB01E3
:10002000A901AA01C201BF01B0017E222420861FBE
:100030001D28A91FA90A052117282420861B162878
:10004000A91FA90A05211E28AA0A290803196B2835
:100050006400A9014210FD3E031C42140318AA01CA
:10006000E7302B070318AB012B0882077A288D286D
:100070009628A728AE28A728AE28A728AE28A72804
:10008000AE28A728AE28A728AE28A728AE28A728DC
:10009000B728C328D528E728F328FF28AB01421C3E
:1000A0007A2A4108031944293508360637063806E6
:1000B0003906031D7D2AC1190800AA01C21136089C
:1000C000E03903190800B61F692836080F39BF0048
:1000D000BF1708000800AB01AA01702AB00A073058
:1000E000300582071A29492972299B29C429ED293B
:1000F000162A422AEC302A07031C4429AB0AB7010E
:10010000B801C101BA010000000000000000FF308A
:10011000B3000000000000000800421CAB0A000011
:10012000000000000230B100B1176F2AAB0A42187C
:10013000AB010000000000000030B200B20DB20DB3
:10014000B20DB20DB2097030B20500000800AB0A62
:10015000031042180314B90DF2284829AB0A421CB7
:10016000B428391CAB01F2283918AB017C2A421C97
:10017000BC28391CAB09BF283918AB090000BA0AE2
:100180003A08AB0745290230AB003908B5004218E0
:10019000AB0135080319C114BF3A031941153508DD
:1001A0007F39903E0318C11508000230AB003908B2
:1001B000B6004218AB0136087039031D41113206F2
:1001C0000319411435083106031D41100800421877
:1001D000EE280230AB003908B7007C2A1830AB009B
:1001E000C21042116E2A4218FA280230AB003908B8
:1001F000B8007C2A1830AB00C21442116E2AAB0A38
:10020000421CAB01C2144215F2283F300102031C0C
:100210006E28C00A810100000A304002031C752AC2
:10022000C001A00AA10AA20AA30AA40AA50AA60A52
:10023000A70A772ABF1F30293F080739003A031D54
:100240003529331C3729BF1D2C2905140515C0017C
:10025000A001BF13851046290510BF1305114529BC
:10026000000000000000000000000000000040301E
:10027000000000000000031945292002031C462944
:100280000510051148294429F2284629472900006C
:100290000800BF1F5F293F080739013A031D642981
:1002A000B31C6629BF1D5B2985140515C001A1017A
:1002B000BF13051046298510BF13051145290000FD
:1002C00000000000000000000000000040300000BE
:1002D00000000000031945292102031C462985104E
:1002E00005114829BF1F88293F080739023A031D15
:1002F0008D29331D8F29BF1D84298614C001A201B9
:10030000BF130515061146298610BF13051145298F
:1003100000000000000000000000000000000000DD
:10032000403000000000031945292202031C462921
:10033000861005114829BF1FB1293F080739033A24
:10034000031DB629B31DB829BF1DAD290615C0016F
:10035000A301BF130515861046290611BF13051109
:10036000452900000000000000000000000000001F
:100370000000403000000000031945292302031C3F
:100380004629061105114829BF1FDA293F080739F8
:10039000043A031DDF29331EE129BF1DD629861526
:1003A000C001A401BF13051506124629BF1386110B
:1003B00005114529000000000000000000000000B9
:1003C000000000004030000000000319452924020D
:1003D000031C4629861105114829BF1F032A3F081F
:1003E0000739053A031D082AB31E0A2ABF1DFF2933
:1003F0000616C001A501BF13051586114629BF13B6
:100400000612051145290000000000000000000050
:1004100000000000000040300000000003194529E2
:100420002502031C4629061205114829BF1F2C2A44
:100430003F080739063A031D312A331F342ABF1DEE
:10044000282A8616C001A601BF13051506134629E2
:10045000BF138612051145290000000000000000AE
:10046000000000000000000000000000000040301C
:1004700000000000031945292602031C46298612A4
:1004800005114829BF1F582A3F080739073A031D9D
:100490005D2A331F602ABF1D542A0617C001A70119
:1004A000BF13051586124629BF13061305114529EA
:1004B000000000000000000000000000000000003C
:1004C0000000000000004030000000000319452932
:1004D0002702031C462906130511482945297D2AB0
:1004E000712A732A0F29742A762A772A782A5028A3
:1004F000792A43297B2AB6286F2AAD28A001A101B9
:0E050000A201A301A401A501A601A701080004
:00000001FF
